:030000000219FDE5
:03000B000200A848
:03002B000201636C
:03005B000202EDB1
:030073000202D3B3
:1000800002030406080C10182030406080040608A3
:100090000C10182030406080A0C000070F1F3F05E3
:1000A000050D050305030302C2AFC0D0C0E0206206
:1000B00017E5256002E473E525F4F58A758B00D217
:1000C00062D0E0D0D0D2AF3285268AC262E526F473
:1000D0006035306803207210758B00D0E0D0D0C23C
:1000E00092C290C291D2AF32C292C290C291206E9F
:1000F0000C206609740AD5E0FDE57E4290758B0000
:10010000D0E0D0D0D2AF32758A00C28DD26201FD6C
:1001100001B7306805206602D29201B73068052029
:100120006602D29101B7306805206602D29001B70D
:10013000C29530680A2066077408D5E0FDD29201A6
:10014000B7C29430680A2066077408D5E0FDD291E2
:1001500001B7C29330680A2066077408D5E0FDD263
:100160009001B7C2AFC2AD53E6EFC0D0C0E0D2D36A
:10017000D2AFC2CEE52A6007207449152A21C4787F
:1001800000790020742EE580307E01F430E702789B
:10019000FF53DACF207E0343DA20307E0343DA10A8
:1001A000C2D8C271E580307E01F430E70279FFC326
:1001B000E89970CB306103752A18207403752A18EA
:1001C000885FD27020740DE52B6004152B21D44379
:1001D000DA01C2D82070024136A85F206102C270E5
:1001E000207431C3E894F0400374F0F8E8C4540F6D
:1001F00028F87984B703024114C313C3138721205D
:100200000802C313200A06C3C898F8411428F850FE
:100210000374FFF8C3E895685003E568F88822E5A1
:100220002D54066011E533C313C31324062522F5AC
:100230002250037522FF852224A824C3E524956457
:100240004002A8648825E5697002417AC3E8AA697A
:100250009A5003E8FAE4F9EAC333FBE56BF45B294F
:10026000400D256AF8E56A6002156A400B417A0A7A
:10027000C3E56A9A5002056A78FF8826C26EC3E514
:100280002694F84002D26EC3E52594404002D26421
:1002900020CF0AD0E0D0D043E610D2AD32C2CF0595
:1002A0003A7801E52A6005307402152AC3E55F94A7
:1002B00001400575620041C9756300756C00E56217
:1002C0002401F56250037562FFD0E0D0D043E61000
:1002D000D2AD32C2AFC0D053E67FC2607591008507
:1002E0005694855795759104D0D0D2AF32C2AF5392
:1002F000E6EFC2ADC0D0C0E0C0F0D2D3D2AFA8FB11
:10030000A9FCC2D8307102615453DACF207E034376
:10031000DA10307E0343DA20D271E580307E01F4BA
:1003200020E702612B88278928A18153DACF207E1C
:100330000343DA20307E0343DA10C2D8C27130742E
:1003400002A16D7800E580307E01F430E702A16DF6
:10035000885FA15553DACF207E0343DA20307E0335
:1003600043DA10C271206102812D53DACF207E035F
:1003700043DA10307E0343DA20C2D8D271885A891A
:100380005BC3E89558F8E99559F97B007E087A0037
:10039000C3E8948CE994005005755E00811F8821A4
:1003A00078A2E6A8216055C3E894C8E994005008F3
:1003B000E4D2E4FB7A0A61FAC3E89468E994015054
:1003C00008E4D2E3FB7A0F61FAC3E894D0E994021F
:1003D0005008E4D2E2FB7A1E61FAC3E894A0E994E3
:1003E000055008E4D2E1FB7A3C61FAC3E89498E94D
:1003F00094085008E4D2E0FB7A787E00C3E8955C6C
:10040000FCE9955DFD30E70AECF42401FCEDF434E1
:1004100000FD755E00C3EC9AED9E5003755E018889
:100420005C895D855A58855B597802A155C3E8956A
:1004300027F8E99528F9307C02A139307B02A139EF
:10044000307A02A1322075028150E9FDE8FC816F0B
:10045000E9C313F9E813F8307902A132E9C313F9BB
:10046000E813F8307802A132E9C313FDE813FC2049
:0E047000612CC3EC941CED940240028186EDD9
:10047E00701EC3EC94C850180529E5297002152981
:10048E00C3E529940A5002A16D755F00D270A16D6B
:10049E00E529600215297888E6F97400207F08782E
:1004AE0096B90302789EE624FAFEE43400FFC3EC0C
:1004BE009EFCED9FFD9208B90310A208500720760E
:1004CE0009D27681D8307602C276A2085016B903C8
:1004DE000DECF42401FCEDF43400FD0204F278007E
:1004EE007900A139B90315EC33FCED33FDC3EC945F
:1004FE000AFCED9400FD50047C007D00C3EC94FFDB
:10050E00ED9400400678FF7900A139EC8575F0A4D2
:10051E00C5F0A2F733F87900400302055578FF794C
:10052E0000020555E9C313F9E813F8307C0EE960B3
:10053E000278FFC3E81338F8E43400F9C3E894FFF7
:10054E00E99400400278FF885FD270206102A16DAD
:10055E00741FF4552F4BF52FC274EB7002D27475C5
:10056E002A18307403752A0A306102A1812074039F
:10057E0053DAFE207403752B06D0F0D0E0D0D0D223
:10058E00AD43E6103279010205B179030205B17966
:10059E000A0205B1791E0205B179640205B179C866
:1005AE000205B17817E4D5E0FDD8FAD9F6227A140F
:1005BE007B780205D87A107B8C0205D87A0D7BB435
:1005CE000205D87A0B7BC80205D87902B27DE4C247
:1005DE0094D5E0FDD291D5E0FDC291D5E0FDD29447
:1005EE00D5E0FDD292E576D5E0FDC2927496D5E0C7
:1005FE00FDD9D9EAF8D5E0FDD8FBDBCEC29422C3F3
:10060E007C007D0075F00005F0EA33FAEB33FB5009
:10061E00F6EB13FBEA13FAC3E9FFE8FEE89AF8E9F2
:10062E009BF95004EFF9EEF8B3EC33FCED33FDD546
:10063E00F0DFEDF9ECF822E889F08A20D2D4F8A99F
:10064E00F07B0030F70B7BFFF42401F8E9F4340063
:10065E00F9E88520F0A4ADF0F8E98520F0A4AFF01C
:10066E00FEED2EF974003FFA7C04C3EA13FAE91387
:10067E00F9E813F8DCF48BF030F70AE8F42401F80B
:10068E00E9F43400F9E889F0C2D4F8A9F02222C3C3
:10069E00E54113F9E54013F8C3E54598F8E54699A9
:1006AE00F9500CC3E89480E994FF40160206D4C3B7
:1006BE00E8947FE9940050030206D4787F79000213
:1006CE0006D4788079FF884A894B22E54A2547F877
:1006DE00E54B3548F9854B20E4300701F43549FAEE
:1006EE0030E709C3EA94F04015020712C3EA940FEB
:1006FE00500302071278FF79FF7A0F020712780073
:10070E0079007AF0C3E5249564500AC374019524E8
:10071E00500B020730E54B20E70E020730E54B3059
:10072E00E706884789488A492278A4E6FAC3E54A4B
:10073E0033F8E54B33F9D145E930E70BC3E8948044
:10074E00E994FF4013E16AC3E8947FE994005002F4
:10075E00E16A787F7900E16A788079FFE820E71511
:10076E00C3E52398F84009C3E894014003020791BA
:10077E007801020791E8F424012523F840030207CB
:10078E009178FF884C2278A5E6FAA848A949D14568
:10079E00E930E70CC3E89401E994FF40160207C55F
:1007AE00C3E894FFE9940050030207C578FF79006F
:1007BE000207C5780179FFE920E715C3E54C98F8E3
:1007CE004009C3E8940140030207EC78010207ECEC
:1007DE00E8F42401254CF840030207EC78FF882446
:1007EE002278FFC26420693D206A12D264C3E541BB
:1007FE00940A4009C3E52594405002C26479A1E7EA
:10080E006023E541601F74FF8541F0848539F03027
:10081E006A0375F005A4F8C5F0600278FFC3E89589
:10082E00675002A867886622C3E5409440E541946C
:10083E0001E5665003140147046002F566220208C2
:10084E004F2275E890227883E6FFE5E820ECF7A8C2
:10085E00BDA9BE0573C3E57394084052757300E9D4
:0D086E00FA79A0E76044EA7007E574601BAA
:10087B0002088AC3E895746010E5745006600C1486
:10088B000208960460F9020896E574F574C3946D3A
:10089B00401B7564C0C394044013756480C39404F7
:1008AB00400B756440C39404400375640075BB062C
:1008BB0022E564F460020564E573B4070375BB10AD
:1008CB0022743279A687F0A4C5F0A2F733F8C3E8F7
:1008DB0095644002A8648822882488258826886726
:1008EB00227540007541F022C2AF75C820A8CCA973
:1008FB00CDAA3A30CF010A75C824D2AFAB3BAC3C82
:10090B00883B893CC3E89BF8E99C206908F9306770
:10091B000241082165AD3D8A3DF9EA9DFA600478F4
:10092B00FF79FFAE3EAF3F8B3E8C3FC3EC9FFCC3CA
:10093B00E99CF542A83BA93CC3E89EF8E99FF9C3A3
:10094B00E54113FBE54013FAE82AF540E93BF54195
:10095B0050067540FF7541FF21AFAA40AB41AC403B
:10096B00AD417E047F02C3EB940440021E1FC3EB18
:10097B00940840021E1FC3ED13FDEC13FCDEF7C3FE
:10098B00EA9CFAEB9DFBEF6009C3E913F9E813F856
:10099B00DFF7EA28FAEB39FB8A408B4150067BFFE5
:1009AB008B408B41C3EB94025002D2673069047FBA
:1009BB000321DA7892E6FFC3E537948240110FC327
:1009CB00E53794A040010FC3EF940640027F057EEC
:1009DB0005E541C4540FF9E541C454F0F8E540C4B2
:1009EB00540F28F8C3E89EFAE99400FB4009C3EAC8
:1009FB009402EB940050047A02E4FB4154AA40ABFE
:100A0B0041EBC4FEEAC4540F4EFCC3EA9CFAEB94D0
:100A1B0000FBC3E813C313F8EA28FAEB3400FB8A94
:100A2B00408B41C3EB94024002C2677805EBC4FED6
:100A3B007B00EAC4540F4EFAC3EA98FA4005C394FC
:100A4B000250027A027892E6FF30600241548552DE
:100A5B0056855357D26043E680C3E49AF8E49BF97A
:100A6B0030670241EEE8FAE9FBD3E913FDE813FC2A
:100A7B0088528953C3EF94036038EF20E00DE82CC4
:100A8B00F8E93DF9ECFAEDFB020AA9E828F8E93997
:100A9B00F9C3E82402F8E93400F97AFE7BFFC3EFCF
:100AAB009403400E8A548B55884E894F8C508D5130
:100ABB006122885489558A4E8B4F8C508D513069E9
:100ACB0020C3E53394034019E542A2E713F8E5553B
:100ADB00F4240138400B20E7087554FFF42401F58A
:100AEB00556122E8FAD3E813FC8852C3EF940360F4
:100AFB0020EF20E007E82CF8ECFA610EE82824023E
:100B0B00F87AFEC3EF940340088A54884E8C5061E8
:100B1B002288548A4E8C50E56BC3335002646BF5BC
:100B2B006B306002612C753402D26043E680E52D98
:100B3B0054066026A840A941C3E913F9E813F8C28B
:100B4B00AF53E67F759100C3E498F594E499F5955E
:100B5B00759104D26043E680D2AF22D26575440012
:100B6B00752000306B03752040020B85D2657544F0
:100B7B0000752040306B03752000D2AF78012067E1
:100B8B0022E52D54066002C265C3E541940540136E
:100B9B007802940540087803940540027806306982
:100BAB0002780A206019E544601530690AC3E53301
:100BBB0094034003D53406D2AFD26C81577134D233
:100BCB00AF0000C2AF206726E541C3FB940F400284
:100BDB007B0FEB240530730123306A0274282062EB
:100BEB000123F93069027982E58BC39940B505443D
:100BFB00E59BF45440B52002814130690A08C3E8F3
:100C0B00940A40010861AE2065026185C26553E616
:100C1B007F7591003067107594007595FE75910482
:100C2B00D26043E6806185AE40AF41C3E49EF5944C
:100C3B00E49FF5958128C3E533940250026185301A
:100C4B0065026185D802815561AEC26C53E67F7532
:100C5B009100855494855595759104854E56854F15
:0E0C6B0057D26043E680D2AFE52D54066008F4
:100C7900206A020533020C91306C0D206B0A206545
:100C8900071581158102150E22780030640530653B
:100C9900027801E53775F007A4F9E5F028F5F0E9E0
:100CA900A2F013A2F113A2F213F537C394785003FB
:100CB900753778C3E53795384008D266C292C29035
:100CC900C29130600281CB855056855157D260431D
:100CD900E68022207D11C2AF754302C294D295D21B
:100CE900AF759F11020EABC2AF754302C294D29386
:100CF900D2AF759F11020EAB307243207D20C2AF77
:100D0900754303900141757E10C290C2933062040D
:100D1900D291A11FD294D2AF759F01020EABC2AF7F
:100D2900754303900141757E10C292C295306204E9
:100D3900D291A13FD294D2AF759F21020EAB207DF3
:100D490017C2AF75430390011CC290306202D29161
:100D5900D2AF759F01020EABC2AF75430390011C60
:100D6900C292306202D291D2AF759F21020EAB209E
:100D79007D11C2AF754304C295D293D2AF759F213D
:100D8900020EABC2AF754304C293D295D2AF759F21
:100D990001020EAB307243207D20C2AF754305902E
:100DA9000130757E20C291C294306204D292A1BBF7
:100DB900D295D2AF759F11020EABC2AF75430590A4
:100DC9000152757E08C291C294306204D290A1DBAF
:100DD900D293D2AF759F11020EAB207D17C2AF75AA
:100DE9004305900112C291306202D292D2AF759F2F
:100DF90011020EABC2AF754305900126C291306254
:100E0900EBD290D2AF759F11020EAB207D11C2AF0C
:100E1900754306C293D294D2AF759F01020EABC23D
:100E2900AF754306C295D294D2AF759F21020EAB1E
:100E3900307242207D20C2AF754301900152757E08
:100E490008C292C295306204D290C157D293D2AFF0
:100E5900759F21020EABC2AF754301900130757EBB
:100E690020C290C293306204D292C177D295D2AF98
:100E7900759F01C1AB207D16C2AF75430190012654
:100E8900C292306202D290D2AF759F21C1ABC2AF7C
:100E9900754301900112C290306202D292D2AF75AD
:100EA9009F01C26622900110757E00C292C290C253
:100EB90091C295C293C294C26222788076FF087665
:100EC900FF0876FF0876FF08760308760408760996
:100ED900087603087601087601788C76010876FF92
:100EE9000876FF0876FF0876FF0876FF087603087C
:100EF90076FF0876FF0876FF0876250876D008760B
:100F0900FA0876FA0876040876FF0876010876006A
:100F190008767A0876FF08760108760108760008CF
:100F29007603227887E6FFC272BF0302D2727888FD
:100F3900E6C394036008C27DE630E102D27DC27E39
:100F49007889E630E102D27EC3EF94026008758E9B
:100F590001D273020F64758E00C273227880E61481
:100F69009000809378A4F67881E6149000809378B5
:100F7900A5F67886E61490008D9378A6F6789CE617
:100F89007538FF75390CB402067538A075390AB47D
:100F9900030675388275390578A3E61490009A938B
:100FA900F569D1AE22227896E6FA7897E6FB788839
:100FB900E6B40305C3EB940EFB307F047A007BFF94
:100FC900C3EB9AFCC3948250027C82757500057547
:100FD900EC8575F0A4C3E5F0947D40F222D27FF14F
:100FE900AF1205A27A007B007C10120598E55F2AF2
:100FF900FA74003BFBDCF37C04C3EB13FBEA13FA42
:10100900DCF7FEC27F120FAF22E5EF20E603752061
:10101900000520903FFFE520146006901DFF146035
:10102900009304600375EF1253D9BF7581C043FF64
:101039008012059375EF0243B203E5B3240420E758
:101049000DF521E5E320E0068521B343E301120E06
:10105900AE7580FF75A40075F19175D47F75900008
:0F10690075A53F75F23F75D50075A60175E2417B
:10107800E4F8F6D8FD756B01120EC3121550789876
:101088008676753001C2AF1205AC1205BC1205A2F6
:101098001205C31205A21205CA1205A21216691278
:1010A80005AC1205AC1205A7C2AF78FA79FA3087F9
:1010B80007D9FBD8F7021C00120F2C120F65120F6C
:1010C800AE120FAF78988676120EAE758850758975
:1010D8001275C82475910475D84075A82275B80290
:1010E80075E690759B80759D0075D10E75BC587519
:1010F800BB0675BA1175E880120593D2AF12084C79
:1011080053DACF207E0343DA20307E0343DA1043DC
:10111800DA01C2D8C2711205ACD2617B037A0CE540
:101128005E70077A0CDB030210B01205A220700370
:101138000210B0C270E55FC3940240E1E52F541F6E
:10114800856160F561B560D5DAD5C26153DACF2023
:101158007E0343DA20307E0343DA10C2D8C27178A6
:10116800A2E67008D274E52F54E0F52FC2757529F0
:10117800001205A7307409C3E529940A4002D27504
:1011880012059878023074027800C3E55F9840F041
:10119800C2AF1205BC1205BC1205BCD2AF1205AC19
:1011A800754D007888E6B403024190120598788C52
:1011B800E6C394015003021290E530C39401500332
:1011C800021290207435C3E55F94FF500302129019
:1011D800C2AF1205D1D2AF1205A7C3E55F94015083
:1011E800EFC2AF1205BC12059D1205BCD2AF1205A5
:1011F800A7C3E55F94FF40E90216EE7F05D27F1290
:101208000FAF1205A7C2AFC27F120FAFAE5FC3E523
:101218005F947FD2AF407B120593C2AF1205D1D243
:10122800AFDFDA120FE6C3EE94057897F61205AC35
:101238001215921216717F0AD27F120FAF1205A7EC
:10124800C2AFC27F120FAFAE5FC3E55F947FD2AF6C
:1012580050E4120593C2AF1205BC12059D1205BCDD
:10126800D2AFDFD4120FE6EE24057896F61205AC5D
:101278001215921216A01205A7120FAFC3E55F94BC
:10128800FF500221CB0216EEC3E55F954D40038562
:101298005F4D1205A778017988E7B403027805C382
:1012A800E55F98400221ABC2AF1205D11205D112F9
:1012B80005D1D2AF1205AC753000E4F531F5320531
:1012C80031E531F470390532789AE67819146012EC
:1012D800783214600D787D14600878FA146003750C
:1012E8003200C3E53298401715327531B4789986C3
:1012F80076C2AF1205D1D2AF789886761205A712BA
:10130800059DE52A700530740201B0780120740249
:101318007806C3E55F9840A77888E6C3940360031E
:101328001205A7E52A70030210B0C2AF120EAEE490
:10133800F522F523F524F525F526F56AD2AF78854B
:10134800E6C333F568E4F545F546F547F548F5494C
:10135800F573F52CF52DF53775730875BB10120567
:1013680093120850E5E820ECFBA8BDA9BEE970017E
:10137800F8887412085475730875BB107887E6FEF0
:101388007602120F2C7887EEF6C2AF7564FF12084A
:10139800CC852264852265852266D2AF75220175C7
:1013A800240175250175260185636C756D017888A2
:1013B800E6B40307C27D307602D27DD268D2697561
:1013C8003300120E14120E391208EC1208F3120828
:1013D800EC1208F31208EC0213EFC2AF120F2CD272
:1013E800AF75730075BB06120B7712069C120C9230
:1013F800120CDC1208F3120B66306D0312069D20E6
:1014080067031207EF306703120836120C92120DA9
:10141800011208F3120B77306D031206D9120C92E1
:10142800120D781208F3120B66306D03120737128B
:101438000C92120D9D1208F3120B77306D031207F0
:1014480094120C92120E141208F3120850120B6622
:10145800120C92120E391208541208F33069322015
:0E1468006B2F85676485676585636C756D0104
:1014760079187A0CC3E53399400CC269D26A8A3569
:101486007564FF021499C3E55F940140030213EFEC
:10149600021516306A1B206B18E535147004C26AF3
:1014A60061E2F535C3E55F940140030213EF0215CF
:1014B60016753600C3E5627882985054307404E598
:1014C6002A604D7888E6B40317207D0520760781CB
:1014D600E630760281E6206B07D26B856764812E43
:1014E60078F0306B058567647820C3E54198500233
:1014F60061EF306B1BC26BC27D307602D27DD26A41
:1015060075351285676461EF0536E55F6002A119DE
:10151600753600C2AF120EAE7887E6FE7602120F5F
:101526002C7887EEF6E4F522F523F524F525F52645
:10153600F568C268D2AF120593120EAE307409C3B5
:10154600E5369405400201B041C2901A0D7820128A
:1015560015D4E520B45A0CA31215D4E520B4A5037E
:10156600021572120EC3121592021591901A037883
:10157600807B0A1215D4A308DBF9901A0F788C7BAE
:10158600181215D4A308DBF9901A2722C2AF121637
:10159600131215ED901A00740E1215D9A3740412C5
:1015A60015D9A374141215D9901A0378807B0A12E0
:1015B60015D8A308DBF9901A0F788C7B181215D86A
:1015C600A308DBF9121626121604901A2722E493B2
:1015D600F622E6438F01538FFD75EF0275B7A575A9
:1015E600B7F1F0538FFE22438F02438F0175EF024E
:1015F60075B7A575B7F1901A0DF0538FFC22901AA6
:101606000D745AB1D9901A0E74A5B1D9227A3079CF
:10161600D07820901A40B1D4E520F709A3DAF72252
:101626007A3079D0901A40E7B1D909A3DAF922AB1A
:1016360077A878BB01027984BB02027985BB0302D5
:101646007986BB04027992BB05027987BB060279CB
:10165600A3BB0702799CBB08027988BB090279897A
:10166600E8F7227C051205ACDCFB22C2AF1205BCF2
:101676001205C31205CA1205D112059D1205BC1228
:1016860005C31205CA1205D112059D1205BC120525
:10169600C31205CA1205D1D2AF22C2AF1205D112AA
:1016A60005CA1205C31205BC12059D1205D1120505
:1016B600CA1205C31205BC12059D1205D11205CA30
:1016C6001205C31205BCD2AF22AE77AF78C2AF12F5
:1016D60005BC1205BC1205BC12059DDEF21205D131
:1016E60012059DDFF8D2AF22D171D169D169757724
:1016F60001757801757900D1CF7C05AD5F1205AC17
:10170600C3ED955F70F5C3E55F9401400AC3E55FDD
:1017160094FF403202172AD135B192D171C2AF750A
:10172600EF12D169DCD50579C3E5799403500280BF
:10173600C6D1690578E5771490009F93F808C3E54C
:101746007898500280AED169D1690577C3E5779460
:101756000A5002809C120EC3B192C2AF75EF12D12D
:011766006919
:0319FD00021012C3
:101A00000E0414FFFFFFFF0304090301015AA5019F
:101A1000FFFFFFFFFF03FFFFFF25D0FAFA04FF01DE
:081A2000007AFF01010003FF41
:101A40002358503335415357232020202020202075
:101A500023424C48454C4923463333302320202031
:101A60002020202020202020202020202020202076
:101C0000C2AFC2D353D9BF7581C043B20343FF8073
:101C1000752438752503B1C975EF0275E24043F1AB
:101C20008053A47F75D400D2877DFA780379E67C4F
:101C300010752200752300901DD67B0675249875BB
:101C400025013087028142208708D8FBD9F9DCF7CB
:101C500081B4308708D8FBD9F9DCF781B4B189E4C5
:101C600093A3C39A6004DDC381B4DBDBB17B600264
:101C7000812B7B08E493FAA3B15CDBF87A30B15C8A
:101C8000752200752300B17BEAFCEBFDC3ED94FEE9
:101C9000400EB17B8A278B28ED30E0048A828B834B
:101CA000B17B7AC270D8C3ED94FE601350CEBD00F4
:101CB00025EC60097520007521FF0200008100A855
:101CC00027A9280809D804D90281D3B17FEA89AAB3
:101CD000F281C50D81A0C3ED94035049EDA2E092BD
:101CE000007AC5C3E5829400E583941C50902000DF
:101CF00010438F02438F0175B7A575B7F1F030001F
:101D00001FA827A9280809438F01538FFDD804D99C
:101D100002A12089AAE275B7A575B7F1F0A3A10DBC
:101D2000538FFC817C7AC1BD030CE493A3FAB140CC
:101D3000DCF8B138817C817EAA22AB23B15CEBFA5E
:101D4000EA6222752608C3E52313F523E52213F57D
:101D50002250066323A0632201D526EAB1C9B1C986
:101D600075260AEAF4200102D287300102C287B147
:101D7000C9C3134002C201D526EB22B17FEAFB2082
:101D80008702A17F308702A184752608AE24AF2583
:101D9000C3EF13FFEE13FEB1CDB1C9C3EA13308711
:101DA000024480FA30E703632201C3E52313F523DD
:101DB000E52213F52250066323A0632201D526D91C
:101DC000E52265236523F52222AE24AF250E0FDE22
:101DD000FEDFFCD20122424C48656C693437316326
:041DE000F3300601D5
:00000001FF
